
 GDI

 Start     Length     Name                   Class
 0001:0000 0265EH     _TEXT                  CODE
 0001:265E 00000H     _GPFIX0                CODE
 0001:265E 00040H     _GPFIX                 CODE
 0001:269E 002C0H     _SORT                  CODE
 0002:0000 00046H     _DATA                  DATA
 0002:0046 00000H     CONST                  CONST
 0002:0046 00000H     _BSS                   BSS

 Origin   Group
 0002:0   DGROUP

 Address   Export                  Alias

 0001:124E ABORTDOC                ABORTDOC
 0001:1BE4 ADDFONTRESOURCE         ADDFONTRESOURCE
 0001:1167 ANIMATEPALETTE          ANIMATEPALETTE
 0001:179C ARC                     ARC
 0001:1E2C BITBLT                  BITBLT
 0001:0166 BRUTE                   BRUTE
 0001:17B8 CHORD                   CHORD
 0001:0180 CLOSEJOB                CLOSEJOB
 0001:1626 CLOSEMETAFILE           CLOSEMETAFILE
 0001:1F20 COMBINERGN              COMBINERGN
 0001:0DB3 CONVERTOUTLINEFONTFILE  CONVERTOUTLINEFONTFILE
 0001:01A7 COPY                    COPY
 0001:15EC COPYMETAFILE            COPYMETAFILE
 0001:1472 CREATEBITMAP            CREATEBITMAP
 0001:148C CREATEBITMAPINDIRECT    CREATEBITMAPINDIRECT
 0001:1458 CREATEBRUSHINDIRECT     CREATEBRUSHINDIRECT
 0001:14CD CREATECOMPATIBLEBITMAP  CREATECOMPATIBLEBITMAP
 0001:12C6 CREATECOMPATIBLEDC      CREATECOMPATIBLEDC
 0001:1306 CREATEDC                CREATEDC
 0001:211F CREATEDIBITMAP          CREATEDIBITMAP
 0001:152B CREATEDIBPATTERNBRUSH   CREATEDIBPATTERNBRUSH
 0001:0FBB CREATEDIBSECTION        CREATEDIBSECTION
 0001:14DB CREATEDISCARDABLEBITMAP  CREATEDISCARDABLEBITMAP
 0001:0229 CREATEELLIPTICRGN       CREATEELLIPTICRGN
 0001:170B CREATEELLIPTICRGNINDIRECT  CREATEELLIPTICRGNINDIRECT
 0001:14E9 CREATEFONT              CREATEFONT
 0001:1511 CREATEFONTINDIRECT      CREATEFONTINDIRECT
 0001:142E CREATEHATCHBRUSH        CREATEHATCHBRUSH
 0001:12D4 CREATEIC                CREATEIC
 0001:160C CREATEMETAFILE          CREATEMETAFILE
 0001:1184 CREATEPALETTE           CREATEPALETTE
 0001:144A CREATEPATTERNBRUSH      CREATEPATTERNBRUSH
 0001:13F8 CREATEPEN               CREATEPEN
 0001:1414 CREATEPENINDIRECT       CREATEPENINDIRECT
 0001:1725 CREATEPOLYGONRGN        CREATEPOLYGONRGN
 0001:1755 CREATEPOLYPOLYGONRGN    CREATEPOLYPOLYGONRGN
 0001:26BF CREATEPQ                CREATEPQ
 0001:02DF CREATERECTRGN           CREATERECTRGN
 0001:1EA8 CREATERECTRGNINDIRECT   CREATERECTRGNINDIRECT
 0001:02F9 CREATEROUNDRECTRGN      CREATEROUNDRECTRGN
 0001:1C12 CREATESCALABLEFONTRESOURCE  CREATESCALABLEFONTRESOURCE
 0001:0306 CREATESOLIDBRUSH        CREATESOLIDBRUSH
 0001:0313 CREATEUSERBITMAP        CREATEUSERBITMAP
 0001:0320 CREATEUSERDISCARDABLEBITMAP  CREATEUSERDISCARDABLEBITMAP
 0001:032D DEATH                   DEATH
 0001:1376 DELETEDC                DELETEDC
 0001:0354 DELETEJOB               DELETEJOB
 0001:1634 DELETEMETAFILE          DELETEMETAFILE
 0001:13EA DELETEOBJECT            DELETEOBJECT
 0001:2899 DELETEPQ                DELETEPQ
 0001:0CFD DELETESPOOLPAGE         DELETESPOOLPAGE
 0001:036E DEVICECOLORMATCH        DEVICECOLORMATCH
 0001:0388 DMBITBLT                DMBITBLT
 0001:0395 DMCOLORINFO             DMCOLORINFO
 0001:0CD6 DMDIBBITS               DMDIBBITS
 0001:03A2 DMENUMDFONTS            DMENUMDFONTS
 0001:03AF DMENUMOBJ               DMENUMOBJ
 0001:0CAF DMEXTTEXTOUT            DMEXTTEXTOUT
 0001:0CBC DMGETCHARWIDTH          DMGETCHARWIDTH
 0001:03BC DMOUTPUT                DMOUTPUT
 0001:03C9 DMPIXEL                 DMPIXEL
 0001:03D6 DMREALIZEOBJECT         DMREALIZEOBJECT
 0001:03E3 DMSCANLR                DMSCANLR
 0001:0CF0 DMSETDIBTODEV           DMSETDIBTODEV
 0001:03F0 DMSTRBLT                DMSTRBLT
 0001:0CC9 DMSTRETCHBLT            DMSTRETCHBLT
 0001:0CE3 DMSTRETCHDIBITS         DMSTRETCHDIBITS
 0001:03FD DMTRANSPOSE             DMTRANSPOSE
 0001:16D1 DPTOLP                  DPTOLP
 0001:178E ELLIPSE                 ELLIPSE
 0001:1270 ENDDOC                  ENDDOC
 0001:125F ENDPAGE                 ENDPAGE
 0001:0431 ENDSPOOLPAGE            ENDSPOOLPAGE
 0001:0D24 ENGINEDELETEFONT        ENGINEDELETEFONT
 0001:0D17 ENGINEENUMERATEFONT     ENGINEENUMERATEFONT
 0001:0DCD ENGINEEXTTEXTOUT        ENGINEEXTTEXTOUT
 0001:0D3E ENGINEGETCHARWIDTH      ENGINEGETCHARWIDTH
 0001:0D58 ENGINEGETGLYPHBMP       ENGINEGETGLYPHBMP
 0001:0D65 ENGINEMAKEFONTDIR       ENGINEMAKEFONTDIR
 0001:0D31 ENGINEREALIZEFONT       ENGINEREALIZEFONT
 0001:0D4B ENGINESETFONTCONTEXT    ENGINESETFONTCONTEXT
 0001:1882 ENUMFONTFAMILIES        ENUMFONTFAMILIES
 0001:185F ENUMFONTS               ENUMFONTS
 0001:1690 ENUMMETAFILE            ENUMMETAFILE
 0001:1835 ENUMOBJECTS             ENUMOBJECTS
 0001:1EC2 EQUALRGN                EQUALRGN
 0001:180C ESCAPE                  ESCAPE
 0001:1E64 EXCLUDECLIPRECT         EXCLUDECLIPRECT
 0001:048C EXCLUDEVISRECT          EXCLUDEVISRECT
 0001:17F0 EXTFLOODFILL            EXTFLOODFILL
 0001:27C7 EXTRACTPQ               EXTRACTPQ
 0001:22FA EXTTEXTOUT              EXTTEXTOUT
 0001:04C0 FASTWINDOWFRAME         FASTWINDOWFRAME
 0001:1F4F FILLRGN                 FILLRGN
 0001:04DA FINALGDIINIT            FINALGDIINIT
 0001:0E90 FIXUPBOGUSPUBLISHERMETAFILE  FIXUPBOGUSPUBLISHERMETAFILE
 0001:17E2 FLOODFILL               FLOODFILL
 0001:1F87 FRAMERGN                FRAMERGN
 0002:0044 FTRAPPING0              FTRAPPING0
 0001:0501 GDIINIT2                GDIINIT2
 0001:050E GDIMOVEBITMAP           GDIMOVEBITMAP
 0001:051B GDIREALIZEPALETTE       GDIREALIZEPALETTE
 0001:0E4F GDISEEGDIDO             GDISEEGDIDO
 0001:0528 GDISELECTPALETTE        GDISELECTPALETTE
 0001:0E5C GDITASKTERMINATION      GDITASKTERMINATION
 0001:1970 GETASPECTRATIOFILTER    GETASPECTRATIOFILTER
 0001:197E GETASPECTRATIOFILTEREX  GETASPECTRATIOFILTEREX
 0001:1914 GETBITMAPBITS           GETBITMAPBITS
 0001:15A8 GETBITMAPDIMENSION      GETBITMAPDIMENSION
 0001:15B6 GETBITMAPDIMENSIONEX    GETBITMAPDIMENSIONEX
 0001:055C GETBKCOLOR              GETBKCOLOR
 0001:0569 GETBKMODE               GETBKMODE
 0001:0C95 GETBOUNDSRECT           GETBOUNDSRECT
 0001:0576 GETBRUSHORG             GETBRUSHORG
 0001:0ED1 GETBRUSHORGEX           GETBRUSHORGEX
 0001:1CE0 GETCHARABCWIDTHS        GETCHARABCWIDTHS
 0001:18A5 GETCHARWIDTH            GETCHARWIDTH
 0001:1E72 GETCLIPBOX              GETCLIPBOX
 0001:059D GETCLIPRGN              GETCLIPRGN
 0001:05AA GETCURLOGFONT           GETCURLOGFONT
 0001:05C4 GETCURRENTPOSITION      GETCURRENTPOSITION
 0001:0EDE GETCURRENTPOSITIONEX    GETCURRENTPOSITIONEX
 0001:0C6E GETDCHOOK               GETDCHOOK
 0001:05D1 GETDCORG                GETDCORG
 0001:05DE GETDCSTATE              GETDCSTATE
 0001:192E GETDEVICECAPS           GETDEVICECAPS
 0001:0FC8 GETDIBCOLORTABLE        GETDIBCOLORTABLE
 0001:223D GETDIBITS               GETDIBITS
 0001:1B88 GETENVIRONMENT          GETENVIRONMENT
 0001:1CA5 GETFONTDATA             GETFONTDATA
 0001:1C44 GETGLYPHOUTLINE         GETGLYPHOUTLINE
 0001:1D2D GETKERNINGPAIRS         GETKERNINGPAIRS
 0001:0612 GETMAPMODE              GETMAPMODE
 0001:1650 GETMETAFILE             GETMETAFILE
 0001:16A7 GETMETAFILEBITS         GETMETAFILEBITS
 0001:19BD GETNEARESTCOLOR         GETNEARESTCOLOR
 0001:11CE GETNEARESTPALETTEINDEX  GETNEARESTPALETTEINDEX
 0001:1956 GETOBJECT               GETOBJECT
 0001:1D13 GETOUTLINETEXTMETRICS   GETOUTLINETEXTMETRICS
 0001:11B1 GETPALETTEENTRIES       GETPALETTEENTRIES
 0001:0653 GETPHYSICALFONTHANDLE   GETPHYSICALFONTHANDLE
 0001:18D8 GETPIXEL                GETPIXEL
 0001:066D GETPOLYFILLMODE         GETPOLYFILLMODE
 0001:0DC0 GETRASTERIZERCAPS       GETRASTERIZERCAPS
 0001:067A GETRELABS               GETRELABS
 0001:1ADC GETRGNBOX               GETRGNBOX
 0001:06A1 GETROP2                 GETROP2
 0001:06AE GETSPOOLJOB             GETSPOOLJOB
 0001:18F8 GETSTOCKOBJECT          GETSTOCKOBJECT
 0001:06CB GETSTRETCHBLTMODE       GETSTRETCHBLTMODE
 0001:11DC GETSYSTEMPALETTEENTRIES  GETSYSTEMPALETTEENTRIES
 0001:11F9 GETSYSTEMPALETTEUSE     GETSYSTEMPALETTEUSE
 0001:06F2 GETTEXTALIGN            GETTEXTALIGN
 0001:1B36 GETTEXTCHARACTEREXTRA   GETTEXTCHARACTEREXTRA
 0001:070C GETTEXTCOLOR            GETTEXTCOLOR
 0001:1AF6 GETTEXTEXTENT           GETTEXTEXTENT
 0001:1B10 GETTEXTEXTENTPOINT      GETTEXTEXTENTPOINT
 0001:1B44 GETTEXTFACE             GETTEXTFACE
 0001:1B6E GETTEXTMETRICS          GETTEXTMETRICS
 0001:0740 GETVIEWPORTEXT          GETVIEWPORTEXT
 0001:0EF8 GETVIEWPORTEXTEX        GETVIEWPORTEXTEX
 0001:074D GETVIEWPORTORG          GETVIEWPORTORG
 0001:0F05 GETVIEWPORTORGEX        GETVIEWPORTORGEX
 0001:075A GETWINDOWEXT            GETWINDOWEXT
 0001:0F12 GETWINDOWEXTEX          GETWINDOWEXTEX
 0001:0767 GETWINDOWORG            GETWINDOWORG
 0001:0F1F GETWINDOWORGEX          GETWINDOWORGEX
 0001:0781 INQUIREVISRGN           INQUIREVISRGN
 0001:2709 INSERTPQ                INSERTPQ
 0001:1E8C INTERSECTCLIPRECT       INTERSECTCLIPRECT
 0001:07A8 INTERSECTVISRECT        INTERSECTVISRECT
 0001:1F95 INVERTRGN               INVERTRGN
 0001:07C2 ISDCCURRENTPALETTE      ISDCCURRENTPALETTE
 0001:07CF ISDCDIRTY               ISDCDIRTY
 0001:0E76 ISGDIOBJECT             ISGDIOBJECT
 0001:010B ISVALIDMETAFILE         ISVALIDMETAFILE
 0001:1D9E LINEDDA                 LINEDDA
 0001:1D4B LINETO                  LINETO
 0001:16EE LPTODP                  LPTODP
 0001:0E83 MAKEOBJECTPRIVATE       MAKEOBJECTPRIVATE
 0001:27C4 MINPQ                   MINPQ
 0001:1D59 MOVETO                  MOVETO
 0001:1D67 MOVETOEX                MOVETOEX
 0001:246C MULDIV                  MULDIV
 0001:1F12 OFFSETCLIPRGN           OFFSETCLIPRGN
 0001:1F04 OFFSETRGN               OFFSETRGN
 0001:19CB OFFSETVIEWPORTORG       OFFSETVIEWPORTORG
 0001:19D9 OFFSETVIEWPORTORGEX     OFFSETVIEWPORTORGEX
 0001:085E OFFSETVISRGN            OFFSETVISRGN
 0001:19F3 OFFSETWINDOWORG         OFFSETWINDOWORG
 0001:1A01 OFFSETWINDOWORGEX       OFFSETWINDOWORGEX
 0001:0878 OPENJOB                 OPENJOB
 0001:1F6B PAINTRGN                PAINTRGN
 0001:1E3A PATBLT                  PATBLT
 0001:17AA PIE                     PIE
 0001:1642 PLAYMETAFILE            PLAYMETAFILE
 0001:166A PLAYMETAFILERECORD      PLAYMETAFILERECORD
 0001:1DB5 POLYGON                 POLYGON
 0001:1D81 POLYLINE                POLYLINE
 0001:1DD2 POLYPOLYGON             POLYPOLYGON
 0001:1DF8 POLYPOLYLINEWOW         POLYPOLYLINEWOW
 0001:1F5D PTINREGION              PTINREGION
 0001:1F79 PTVISIBLE               PTVISIBLE
 0001:0FE2 QUERYABORT              QUERYABORT
 0001:0907 QUERYJOB                QUERYJOB
 0001:0921 REALIZEDEFAULTPALETTE   REALIZEDEFAULTPALETTE
 0001:17D4 RECTANGLE               RECTANGLE
 0001:1ED0 RECTINREGION            RECTINREGION
 0001:0EAA RECTINREGION_EHH        RECTINREGION_EHH
 0001:1EEA RECTVISIBLE             RECTVISIBLE
 0001:0E9D RECTVISIBLE_EHH         RECTVISIBLE_EHH
 0001:1BFB REMOVEFONTRESOURCE      REMOVEFONTRESOURCE
 0001:13A0 RESETDC                 RESETDC
 0001:1207 RESIZEPALETTE           RESIZEPALETTE
 0001:1384 RESTOREDC               RESTOREDC
 0001:0989 RESTOREVISRGN           RESTOREVISRGN
 0001:0996 RESURRECTION            RESURRECTION
 0001:17C6 ROUNDRECT               ROUNDRECT
 0001:1392 SAVEDC                  SAVEDC
 0001:09CA SAVEVISRGN              SAVEVISRGN
 0001:1A8C SCALEVIEWPORTEXT        SCALEVIEWPORTEXT
 0001:1A9A SCALEVIEWPORTEXTEX      SCALEVIEWPORTEXTEX
 0001:1AB4 SCALEWINDOWEXT          SCALEWINDOWEXT
 0001:1AC2 SCALEWINDOWEXTEX        SCALEWINDOWEXTEX
 0001:09FE SCANLR                  SCANLR
 0001:0CA2 SELECTBITMAP            SELECTBITMAP
 0001:1E9A SELECTCLIPRGN           SELECTCLIPRGN
 0001:1FA3 SELECTOBJECT            SELECTOBJECT
 0001:0A25 SELECTVISRGN            SELECTVISRGN
 0001:12AC SETABORTPROC            SETABORTPROC
 0001:193C SETBITMAPBITS           SETBITMAPBITS
 0001:1580 SETBITMAPDIMENSION      SETBITMAPDIMENSION
 0001:158E SETBITMAPDIMENSIONEX    SETBITMAPDIMENSIONEX
 0001:1FBF SETBKCOLOR              SETBKCOLOR
 0001:1FCF SETBKMODE               SETBKMODE
 0001:0C88 SETBOUNDSRECT           SETBOUNDSRECT
 0001:1E48 SETBRUSHORG             SETBRUSHORG
 0001:0C61 SETDCHOOK               SETDCHOOK
 0001:0A73 SETDCORG                SETDCORG
 0001:0A80 SETDCSTATE              SETDCSTATE
 0001:0A8D SETDCSTATUS             SETDCSTATUS
 0001:0FD5 SETDIBCOLORTABLE        SETDIBCOLORTABLE
 0001:20BF SETDIBITS               SETDIBITS
 0001:21B7 SETDIBITSTODEVICE       SETDIBITSTODEVICE
 0001:1BBE SETENVIRONMENT          SETENVIRONMENT
 0001:0C7B SETHOOKFLAGS            SETHOOKFLAGS
 0001:1A1B SETMAPMODE              SETMAPMODE
 0001:1998 SETMAPPERFLAGS          SETMAPPERFLAGS
 0001:16B5 SETMETAFILEBITS         SETMETAFILEBITS
 0001:16C3 SETMETAFILEBITSBETTER   SETMETAFILEBITSBETTER
 0001:0E69 SETOBJECTOWNER          SETOBJECTOWNER
 0001:1215 SETPALETTEENTRIES       SETPALETTEENTRIES
 0001:18E6 SETPIXEL                SETPIXEL
 0001:204E SETPOLYFILLMODE         SETPOLYFILLMODE
 0001:1F41 SETRECTRGN              SETRECTRGN
 0001:0B0F SETRELABS               SETRELABS
 0001:200C SETROP2                 SETROP2
 0001:202D SETSTRETCHBLTMODE       SETSTRETCHBLTMODE
 0001:1232 SETSYSTEMPALETTEUSE     SETSYSTEMPALETTEUSE
 0001:1FF0 SETTEXTALIGN            SETTEXTALIGN
 0001:15DE SETTEXTCHARACTEREXTRA   SETTEXTCHARACTEREXTRA
 0001:1FB1 SETTEXTCOLOR            SETTEXTCOLOR
 0001:15D0 SETTEXTJUSTIFICATION    SETTEXTJUSTIFICATION
 0001:1A64 SETVIEWPORTEXT          SETVIEWPORTEXT
 0001:1A72 SETVIEWPORTEXTEX        SETVIEWPORTEXTEX
 0001:2097 SETVIEWPORTORG          SETVIEWPORTORG
 0001:20A5 SETVIEWPORTORGEX        SETVIEWPORTORGEX
 0001:1A3C SETWINDOWEXT            SETWINDOWEXT
 0001:1A4A SETWINDOWEXTEX          SETWINDOWEXTEX
 0001:206F SETWINDOWORG            SETWINDOWORG
 0001:207D SETWINDOWORGEX          SETWINDOWORGEX
 0001:0BB8 SHRINKGDIHEAP           SHRINKGDIHEAP
 0001:28AF SIZEPQ                  SIZEPQ
 0001:0D0A SPOOLFILE               SPOOLFILE
 0001:1281 STARTDOC                STARTDOC
 0001:129E STARTPAGE               STARTPAGE
 0001:0BC5 STARTSPOOLPAGE          STARTSPOOLPAGE
 0001:1E1E STRETCHBLT              STRETCHBLT
 0001:229D STRETCHDIBITS           STRETCHDIBITS
 0001:233A TEXTOUT                 TEXTOUT
 0001:0EB7 UNICODETOANSI           UNICODETOANSI
 0001:1E56 UNREALIZEOBJECT         UNREALIZEOBJECT
 0001:1240 UPDATECOLORS            UPDATECOLORS
 0001:002F WEP                     WEP
 0001:0C3A WRITEDIALOG             WRITEDIALOG
 0001:0C47 WRITESPOOL              WRITESPOOL
 0001:265E __GP                    __GP

  Address         Publics by Name

 0001:124E       ABORTDOC
 0001:1BE4       ADDFONTRESOURCE
 0001:1167       ANIMATEPALETTE
 0001:179C       ARC
 0001:1E2C       BITBLT
 0001:0C54       BITMAPBITS
 0001:0166       BRUTE
 0001:003B       CheckStockObject
 0001:17B8       CHORD
 0001:0180       CLOSEJOB
 0001:1626       CLOSEMETAFILE
 0001:23AA       CLP0TEXT
 0001:23BE       CLPexitTEXT
 0001:2420       CLPSTRATOM0TEXT
 0001:2422       CLPSTRATOMTEXT
 0001:242E       CLPSZ0TEXT
 0001:2434       CLPSZTEXT
 0001:23B0       CLPTEXT
 0001:1F20       COMBINERGN
 0001:0DB3       CONVERTOUTLINEFONTFILE
 0001:01A7       COPY
 0001:15EC       COPYMETAFILE
 0001:1472       CREATEBITMAP
 0001:148C       CREATEBITMAPINDIRECT
 0001:1458       CREATEBRUSHINDIRECT
 0001:14CD       CREATECOMPATIBLEBITMAP
 0001:12C6       CREATECOMPATIBLEDC
 0001:1306       CREATEDC
 0001:211F       CREATEDIBITMAP
 0001:152B       CREATEDIBPATTERNBRUSH
 0001:0FBB       CREATEDIBSECTION
 0001:14DB       CREATEDISCARDABLEBITMAP
 0001:0229       CREATEELLIPTICRGN
 0001:170B       CREATEELLIPTICRGNINDIRECT
 0001:14E9       CREATEFONT
 0001:1511       CREATEFONTINDIRECT
 0001:142E       CREATEHATCHBRUSH
 0001:12D4       CREATEIC
 0001:160C       CREATEMETAFILE
 0001:1184       CREATEPALETTE
 0001:144A       CREATEPATTERNBRUSH
 0001:13F8       CREATEPEN
 0001:1414       CREATEPENINDIRECT
 0001:1725       CREATEPOLYGONRGN
 0001:1755       CREATEPOLYPOLYGONRGN
 0001:26BF       CREATEPQ
 0001:02DF       CREATERECTRGN
 0001:1EA8       CREATERECTRGNINDIRECT
 0001:02F9       CREATEROUNDRECTRGN
 0001:1C12       CREATESCALABLEFONTRESOURCE
 0001:0306       CREATESOLIDBRUSH
 0001:0313       CREATEUSERBITMAP
 0001:0320       CREATEUSERDISCARDABLEBITMAP
 0001:032D       DEATH
 0001:1376       DELETEDC
 0001:0354       DELETEJOB
 0001:1634       DELETEMETAFILE
 0001:13EA       DELETEOBJECT
 0001:2899       DELETEPQ
 0001:0CFD       DELETESPOOLPAGE
 0001:036E       DEVICECOLORMATCH
 0001:1140       DIB_Validate_Huge_Pointer
 0001:111A       DIB_Validate_Pointer
 0001:0388       DMBITBLT
 0001:0395       DMCOLORINFO
 0001:0CD6       DMDIBBITS
 0001:03A2       DMENUMDFONTS
 0001:03AF       DMENUMOBJ
 0001:0CAF       DMEXTTEXTOUT
 0001:0CBC       DMGETCHARWIDTH
 0001:03BC       DMOUTPUT
 0001:03C9       DMPIXEL
 0001:03D6       DMREALIZEOBJECT
 0001:03E3       DMSCANLR
 0001:0CF0       DMSETDIBTODEV
 0001:03F0       DMSTRBLT
 0001:0CC9       DMSTRETCHBLT
 0001:0CE3       DMSTRETCHDIBITS
 0001:03FD       DMTRANSPOSE
 0001:16D1       DPTOLP
 0001:178E       ELLIPSE
 0001:1270       ENDDOC
 0001:125F       ENDPAGE
 0001:0431       ENDSPOOLPAGE
 0001:0D24       ENGINEDELETEFONT
 0001:0D17       ENGINEENUMERATEFONT
 0001:0DCD       ENGINEEXTTEXTOUT
 0001:0D3E       ENGINEGETCHARWIDTH
 0001:0D58       ENGINEGETGLYPHBMP
 0001:0D65       ENGINEMAKEFONTDIR
 0001:0D31       ENGINEREALIZEFONT
 0001:0D4B       ENGINESETFONTCONTEXT
 0001:1882       ENUMFONTFAMILIES
 0001:185F       ENUMFONTS
 0001:1690       ENUMMETAFILE
 0001:1835       ENUMOBJECTS
 0001:1EC2       EQUALRGN
 0001:2455       ErrorStrPtrTEXT
 0001:180C       ESCAPE
 0001:1E64       EXCLUDECLIPRECT
 0001:048C       EXCLUDEVISRECT
 0001:17F0       EXTFLOODFILL
 0001:27C7       EXTRACTPQ
 0001:22FA       EXTTEXTOUT
 0001:269E       farGDIGlobalAlloc
 0001:04C0       FASTWINDOWFRAME
 0001:1F4F       FILLRGN
 0001:04DA       FINALGDIINIT
 0001:0E90       FIXUPBOGUSPUBLISHERMETAFILE
 0001:17E2       FLOODFILL
 0001:1F87       FRAMERGN
 0002:0044       FTRAPPING0
 0001:0000       GDI16
 0001:0501       GDIINIT2
 0001:050E       GDIMOVEBITMAP
 0001:051B       GDIREALIZEPALETTE
 0001:0E4F       GDISEEGDIDO
 0001:0528       GDISELECTPALETTE
 0001:0E5C       GDITASKTERMINATION
 0001:1970       GETASPECTRATIOFILTER
 0001:197E       GETASPECTRATIOFILTEREX
 0001:1914       GETBITMAPBITS
 0001:15A8       GETBITMAPDIMENSION
 0001:15B6       GETBITMAPDIMENSIONEX
 0001:055C       GETBKCOLOR
 0001:0569       GETBKMODE
 0001:0C95       GETBOUNDSRECT
 0001:0576       GETBRUSHORG
 0001:0ED1       GETBRUSHORGEX
 0001:1CE0       GETCHARABCWIDTHS
 0001:18A5       GETCHARWIDTH
 0001:1E72       GETCLIPBOX
 0001:059D       GETCLIPRGN
 0001:05AA       GETCURLOGFONT
 0001:05C4       GETCURRENTPOSITION
 0001:0EDE       GETCURRENTPOSITIONEX
 0001:0C6E       GETDCHOOK
 0001:05D1       GETDCORG
 0001:05DE       GETDCSTATE
 0001:192E       GETDEVICECAPS
 0001:0FC8       GETDIBCOLORTABLE
 0001:223D       GETDIBITS
 0001:1B88       GETENVIRONMENT
 0001:1CA5       GETFONTDATA
 0001:1C44       GETGLYPHOUTLINE
 0001:1D2D       GETKERNINGPAIRS
 0001:2885       GetLesserChild
 0001:0612       GETMAPMODE
 0001:1650       GETMETAFILE
 0001:16A7       GETMETAFILEBITS
 0001:27C9       GetMinPQ
 0000:0000  Imp  GETMODULEFILENAME    (KERNEL.49)
 0000:0000  Imp  GETMODULEHANDLE      (KERNEL.47)
 0001:19BD       GETNEARESTCOLOR
 0001:11CE       GETNEARESTPALETTEINDEX
 0001:1956       GETOBJECT
 0001:1D13       GETOUTLINETEXTMETRICS
 0001:11B1       GETPALETTEENTRIES
 0001:0653       GETPHYSICALFONTHANDLE
 0001:18D8       GETPIXEL
 0001:066D       GETPOLYFILLMODE
 0001:0DC0       GETRASTERIZERCAPS
 0001:067A       GETRELABS
 0001:1ADC       GETRGNBOX
 0001:06A1       GETROP2
 0001:06AE       GETSPOOLJOB
 0001:18F8       GETSTOCKOBJECT
 0001:06CB       GETSTRETCHBLTMODE
 0001:11DC       GETSYSTEMPALETTEENTRIES
 0001:11F9       GETSYSTEMPALETTEUSE
 0001:06F2       GETTEXTALIGN
 0001:1B36       GETTEXTCHARACTEREXTRA
 0001:070C       GETTEXTCOLOR
 0001:1AF6       GETTEXTEXTENT
 0001:1B10       GETTEXTEXTENTPOINT
 0001:1B44       GETTEXTFACE
 0001:1B6E       GETTEXTMETRICS
 0001:0740       GETVIEWPORTEXT
 0001:0EF8       GETVIEWPORTEXTEX
 0001:074D       GETVIEWPORTORG
 0001:0F05       GETVIEWPORTORGEX
 0001:075A       GETWINDOWEXT
 0001:0F12       GETWINDOWEXTEX
 0001:0767       GETWINDOWORG
 0001:0F1F       GETWINDOWORGEX
 0001:2354       GHANDLE0TEXT
 0001:2358       GHANDLETEXT
 0000:0000  Imp  GlobalAlloc          (KERNEL.15)
 0000:0000  Imp  GlobalFree           (KERNEL.17)
 0000:0000  Imp  GlobalHandle         (KERNEL.21)
 0000:0000  Imp  GlobalLock           (KERNEL.18)
 0000:0000  Imp  GlobalReAlloc        (KERNEL.16)
 0000:0000  Imp  GLOBALUNLOCK         (KERNEL.19)
 0000:0000  Imp  HandleParamError     (KERNEL.327)
 0001:0E42       IABORTDOC
 0001:24D4       IAddFontResource
 0001:013F       IANIMATEPALETTE
 0001:014C       IARC
 0001:0159       IBITBLT
 0001:0173       ICHORD
 0001:00BD       ICLOSEMETAFILE
 0001:018D       ICOMBINERGN
 0001:019A       ICOMPATIBLEBITMAP
 0001:00CA       ICOPYMETAFILE
 0001:01B4       ICREATEBITMAP
 0001:01C1       ICREATEBITMAPINDIRECT
 0001:01CE       ICREATEBRUSHINDIRECT
 0001:01DB       ICREATECOMPATIBLEBITMAP
 0001:01E8       ICREATECOMPATIBLEDC
 0001:01F5       ICREATEDC
 0001:0202       ICREATEDIBITMAP
 0001:2614       ICreateDIBPatternBrush
 0001:021C       ICREATEDISCARDABLEBITMAP
 0001:0236       ICREATEELLIPTICRGNINDIRECT
 0001:0243       ICREATEFONT
 0001:0250       ICREATEFONTINDIRECT
 0001:025D       ICREATEHATCHBRUSH
 0001:026A       ICREATEIC
 0001:00D7       ICREATEMETAFILE
 0001:0277       ICREATEPALETTE
 0001:0284       ICREATEPATTERNBRUSH
 0001:0291       ICREATEPEN
 0001:029E       ICREATEPENINDIRECT
 0001:02AB       ICREATEPOLYGONRGN
 0001:02B8       ICREATEPOLYPOLYGONRGN
 0001:02C5       ICREATEREALBITMAP
 0001:02D2       ICREATEREALBITMAPINDIRECT
 0001:02EC       ICREATERECTRGNINDIRECT
 0001:0D99       ICREATESCALABLEFONTRESOURCE
 0001:033A       IDELETEABOVELINEFONTS
 0001:0347       IDELETEDC
 0001:00E4       IDELETEMETAFILE
 0001:0361       IDELETEOBJECT
 0001:037B       IDEVICEMODE
 0001:040A       IDPTOLP
 0001:0417       IDPXLATE
 0001:0424       IELLIPSE
 0001:0E0E       IENDDOC
 0001:0E28       IENDPAGE
 0001:043E       IENUMCALLBACK
 0001:0DDA       IENUMFONTFAMILIES
 0001:044B       IENUMFONTS
 0001:00FE       IENUMMETAFILE
 0001:0458       IENUMOBJECTS
 0001:0465       IEQUALRGN
 0001:0472       IESCAPE
 0001:047F       IEXCLUDECLIPRECT
 0001:0499       IEXTDEVICEMODE
 0001:04A6       IEXTFLOODFILL
 0001:04B3       IEXTTEXTOUT
 0001:04CD       IFILLRGN
 0001:04E7       IFLOODFILL
 0001:04F4       IFRAMERGN
 0001:0535       IGETASPECTRATIOFILTER
 0001:0FAE       IGETASPECTRATIOFILTEREX
 0001:0542       IGETBITMAPBITS
 0001:054F       IGETBITMAPDIMENSION
 0001:0EC4       IGETBITMAPDIMENSIONEX
 0001:0D72       IGETCHARABCWIDTHS
 0001:0583       IGETCHARWIDTH
 0001:0590       IGETCLIPBOX
 0001:05B7       IGETCURRENTOBJECT
 0001:05EB       IGETDEVICECAPS
 0001:05F8       IGETDIBITS
 0001:0605       IGETENVIRONMENT
 0001:0DA6       IGETFONTDATA
 0001:0D8C       IGETGLYPHOUTLINE
 0001:0DE7       IGETKERNINGPAIRS
 0001:00F1       IGETMETAFILE
 0001:0062       IGetMetafileBits
 0001:061F       IGETNEARESTCOLOR
 0001:062C       IGETNEARESTPALETTEINDEX
 0001:0639       IGETOBJECT
 0001:0D7F       IGETOUTLINETEXTMETRICS
 0001:0646       IGETPALETTEENTRIES
 0001:0660       IGETPIXEL
 0001:0687       IGETREGIONDATA
 0001:0694       IGETRGNBOX
 0001:06BB       IGETSTOCKOBJECT
 0001:06D8       IGETSYSTEMPALETTEENTRIES
 0001:06E5       IGETSYSTEMPALETTEUSE
 0001:06FF       IGETTEXTCHARACTEREXTRA
 0001:0719       IGETTEXTEXTENT
 0001:0EEB       IGETTEXTEXTENTPOINT
 0001:0726       IGETTEXTFACE
 0001:0733       IGETTEXTMETRICS
 0001:0774       IGSV
 0001:078E       IINTERNALCREATEDC
 0001:079B       IINTERSECTCLIPRECT
 0001:07B5       IINVERTRGN
 0001:07DC       ILINEDDA
 0001:07E9       ILINETO
 0001:07F6       ILPTODP
 0001:0803       ILVBUNION
 0001:0810       IMFDRAWTEXT
 0001:081D       IMOVETO
 0001:0F87       IMOVETOEX
 0001:0781       INQUIREVISRGN
 0001:2709       INSERTPQ
 0001:1E8C       INTERSECTCLIPRECT
 0001:07A8       INTERSECTVISRECT
 0001:238C       Inval_Param_TEXT
 0001:1F95       INVERTRGN
 0001:082A       IOFFSETCLIPRGN
 0001:0837       IOFFSETORG
 0001:0844       IOFFSETRGN
 0001:0851       IOFFSETVIEWPORTORG
 0001:0F2C       IOFFSETVIEWPORTORGEX
 0001:086B       IOFFSETWINDOWORG
 0001:0F39       IOFFSETWINDOWORGEX
 0001:0885       IPAINTRGN
 0001:0892       IPATBLT
 0001:089F       IPIE
 0001:08AC       IPIXTOLINE
 0001:0118       IPLAYMETAFILE
 0001:0125       IPLAYMETAFILERECORD
 0001:08B9       IPOLYGON
 0001:08C6       IPOLYLINE
 0001:08D3       IPOLYPOLYGON
 0001:08E0       IPOLYPOLYLINEWOW
 0001:08ED       IPTINREGION
 0001:08FA       IPTVISIBLE
 0001:0914       IRCOS
 0001:092E       IRECTANGLE
 0001:093B       IRECTINREGION
 0001:0948       IRECTSTUFF
 0001:0955       IRECTVISIBLE
 0001:2594       IRemoveFontResource
 0001:0DF4       IRESETDC
 0001:096F       IRESIZEPALETTE
 0001:097C       IRESTOREDC
 0001:09A3       IROUNDRECT
 0001:09B0       IRSIN
 0001:09BD       ISAVEDC
 0000:0000  Imp  IsBadHugeReadPtr     (KERNEL.346)
 0000:0000  Imp  IsBadHugeWritePtr    (KERNEL.347)
 0000:0000  Imp  IsBadReadPtr         (KERNEL.334)
 0000:0000  Imp  IsBadWritePtr        (KERNEL.335)
 0001:09D7       ISCALEEXT
 0001:09E4       ISCALEVIEWPORTEXT
 0001:0F94       ISCALEVIEWPORTEXTEX
 0001:09F1       ISCALEWINDOWEXT
 0001:0FA1       ISCALEWINDOWEXTEX
 0001:07C2       ISDCCURRENTPALETTE
 0001:07CF       ISDCDIRTY
 0001:0A0B       ISELECTCLIPRGN
 0001:0A18       ISELECTOBJECT
 0001:0E35       ISETABORTPROC
 0001:0A32       ISETBITMAPBITS
 0001:0A3F       ISETBITMAPDIMENSION
 0001:0F46       ISETBITMAPDIMENSIONEX
 0001:0A4C       ISETBKCOLOR
 0001:0A59       ISETBKMODE
 0001:0A66       ISETBRUSHORG
 0001:0A9A       ISETDIBITS
 0001:0AA7       ISETDIBITSTODEVICE
 0001:0AB4       ISETENVIRONMENT
 0001:0AC1       ISETMAPMODE
 0001:0ACE       ISETMAPPERFLAGS
 0001:0085       ISetMetafileBits
 0001:009B       ISetMetafileBitsBetter
 0001:0ADB       ISETPALETTEENTRIES
 0001:0AE8       ISETPIXEL
 0001:0AF5       ISETPOLYFILLMODE
 0001:0B02       ISETRECTRGN
 0001:0B1C       ISETROP2
 0001:0B29       ISETSTRETCHBLTMODE
 0001:0B36       ISETSYSTEMPALETTEUSE
 0001:0B43       ISETTEXTALIGN
 0001:0B50       ISETTEXTCHARACTEREXTRA
 0001:0B5D       ISETTEXTCOLOR
 0001:0B6A       ISETTEXTJUSTIFICATION
 0001:0B77       ISETVIEWPORTEXT
 0001:0F53       ISETVIEWPORTEXTEX
 0001:0B84       ISETVIEWPORTORG
 0001:0F60       ISETVIEWPORTORGEX
 0001:0B91       ISETWINDOWEXT
 0001:0F6D       ISETWINDOWEXTEX
 0001:0B9E       ISETWINDOWORG
 0001:0F7A       ISETWINDOWORGEX
 0001:0BAB       ISETWINVIEWEXT
 0001:0E76       ISGDIOBJECT
 0001:0E01       ISTARTDOC
 0001:0E1B       ISTARTPAGE
 0001:0BD2       ISTRETCHBLT
 0001:0BDF       ISTRETCHDIBITS
 0001:0BEC       ISTUFFINREGION
 0001:0BF9       ISTUFFVISIBLE
 0001:010B       ISVALIDMETAFILE
 0001:0C06       ITEXTOUT
 0001:0C13       IUNREALIZEOBJECT
 0001:0C20       IUPDATECOLORS
 0001:0C2D       IWORDSET
 0001:1D9E       LINEDDA
 0001:1D4B       LINETO
 0000:0000  Imp  LocalInit            (KERNEL.4)
 0000:0000  Imp  LOCKRESOURCE         (KERNEL.62)
 0001:2394       LP0TEXT
 0001:23C7       LPBUF0TEXT
 0001:23F6       LPBUFexitTEXT
 0001:23CD       LPBUFTEXT
 0001:236C       LPFN0TEXT
 0001:2372       LPFNTEXT
 0001:239A       LPTEXT
 0001:16EE       LPTODP
 0001:0E83       MAKEOBJECTPRIVATE
 0001:27C4       MINPQ
 0001:1D59       MOVETO
 0001:1D67       MOVETOEX
 0001:246C       MULDIV
 0001:1F12       OFFSETCLIPRGN
 0001:1F04       OFFSETRGN
 0001:19CB       OFFSETVIEWPORTORG
 0001:19D9       OFFSETVIEWPORTORGEX
 0001:085E       OFFSETVISRGN
 0001:19F3       OFFSETWINDOWORG
 0001:1A01       OFFSETWINDOWORGEX
 0001:0878       OPENJOB
 0001:1F6B       PAINTRGN
 0001:1E3A       PATBLT
 0001:17AA       PIE
 0001:1642       PLAYMETAFILE
 0001:166A       PLAYMETAFILERECORD
 0001:1DB5       POLYGON
 0001:1D81       POLYLINE
 0001:1DD2       POLYPOLYGON
 0001:1DF8       POLYPOLYLINEWOW
 0001:1F5D       PTINREGION
 0001:1F79       PTVISIBLE
 0001:0FE2       QUERYABORT
 0001:0907       QUERYJOB
 0001:0921       REALIZEDEFAULTPALETTE
 0001:17D4       RECTANGLE
 0001:1ED0       RECTINREGION
 0001:0EAA       RECTINREGION_EHH
 0001:1EEA       RECTVISIBLE
 0001:0E9D       RECTVISIBLE_EHH
 0001:1BFB       REMOVEFONTRESOURCE
 0001:13A0       RESETDC
 0001:1207       RESIZEPALETTE
 0001:1384       RESTOREDC
 0001:0989       RESTOREVISRGN
 0001:0996       RESURRECTION
 0001:17C6       ROUNDRECT
 0001:1392       SAVEDC
 0001:09CA       SAVEVISRGN
 0001:1A8C       SCALEVIEWPORTEXT
 0001:1A9A       SCALEVIEWPORTEXTEX
 0001:1AB4       SCALEWINDOWEXT
 0001:1AC2       SCALEWINDOWEXTEX
 0001:09FE       SCANLR
 0001:0CA2       SELECTBITMAP
 0001:1E9A       SELECTCLIPRGN
 0001:1FA3       SELECTOBJECT
 0001:0A25       SELECTVISRGN
 0001:12AC       SETABORTPROC
 0001:193C       SETBITMAPBITS
 0001:1580       SETBITMAPDIMENSION
 0001:158E       SETBITMAPDIMENSIONEX
 0001:1FBF       SETBKCOLOR
 0001:1FCF       SETBKMODE
 0001:0C88       SETBOUNDSRECT
 0001:1E48       SETBRUSHORG
 0001:0C61       SETDCHOOK
 0001:0A73       SETDCORG
 0001:0A80       SETDCSTATE
 0001:0A8D       SETDCSTATUS
 0001:0FD5       SETDIBCOLORTABLE
 0001:20BF       SETDIBITS
 0001:21B7       SETDIBITSTODEVICE
 0001:245B       SETEMPTYTEXT
 0001:1BBE       SETENVIRONMENT
 0001:0C7B       SETHOOKFLAGS
 0001:1A1B       SETMAPMODE
 0001:1998       SETMAPPERFLAGS
 0001:16B5       SETMETAFILEBITS
 0001:16C3       SETMETAFILEBITSBETTER
 0001:0E69       SETOBJECTOWNER
 0001:1215       SETPALETTEENTRIES
 0001:18E6       SETPIXEL
 0001:204E       SETPOLYFILLMODE
 0001:1F41       SETRECTRGN
 0001:0B0F       SETRELABS
 0001:200C       SETROP2
 0001:202D       SETSTRETCHBLTMODE
 0001:1232       SETSYSTEMPALETTEUSE
 0001:1FF0       SETTEXTALIGN
 0001:15DE       SETTEXTCHARACTEREXTRA
 0001:1FB1       SETTEXTCOLOR
 0001:15D0       SETTEXTJUSTIFICATION
 0001:1A64       SETVIEWPORTEXT
 0001:1A72       SETVIEWPORTEXTEX
 0001:2097       SETVIEWPORTORG
 0001:20A5       SETVIEWPORTORGEX
 0001:1A3C       SETWINDOWEXT
 0001:1A4A       SETWINDOWEXTEX
 0001:206F       SETWINDOWORG
 0001:207D       SETWINDOWORGEX
 0001:0BB8       SHRINKGDIHEAP
 0001:28AF       SIZEPQ
 0001:0D0A       SPOOLFILE
 0001:1281       STARTDOC
 0001:129E       STARTPAGE
 0001:0BC5       STARTSPOOLPAGE
 0001:1E1E       STRETCHBLT
 0001:229D       STRETCHDIBITS
 0001:27A2       TestShuffle
 0001:233A       TEXTOUT
 0001:0EB7       UNICODETOANSI
 0001:1E56       UNREALIZEOBJECT
 0001:1240       UPDATECOLORS
 0001:0FF4       ValidateDIBHeader
 0001:1098       ValidateDIBSize
 0001:246C       VEndTEXT
 0001:2354       VStartTEXT
 0001:002F       WEP
 0000:0000  Imp  WOW16Call            (KERNEL.500)
 0001:0132       WOWADDFONTRESOURCE
 0001:020F       WOWCREATEDIBPATTERNBRUSH
 0001:0962       WOWREMOVEFONTRESOURCE
 0001:0C3A       WRITEDIALOG
 0001:0C47       WRITESPOOL
 0000:0000  Abs  __acrtused
 0001:265E       __GP
 0000:0000  Imp  __MOD_COMMDLG        (KERNEL.532)
 0000:0000  Imp  __MOD_DGDI           (KERNEL.525)
 0000:0000  Imp  __MOD_DKERNEL        (KERNEL.521)
 0000:0000  Imp  __MOD_DUSER          (KERNEL.523)
 0000:0000  Imp  __MOD_GDI            (KERNEL.524)
 0000:0000  Imp  __MOD_KERNEL         (KERNEL.520)
 0000:0000  Imp  __MOD_KEYBOARD       (KERNEL.526)
 0000:0000  Imp  __MOD_MMEDIA         (KERNEL.531)
 0000:0000  Imp  __MOD_SHELL          (KERNEL.528)
 0000:0000  Imp  __MOD_SOUND          (KERNEL.527)
 0000:0000  Imp  __MOD_TOOLHELP       (KERNEL.530)
 0000:0000  Imp  __MOD_USER           (KERNEL.522)
 0000:0000  Imp  __MOD_WINSOCK        (KERNEL.529)

  Address         Publics by Value

 0000:0000  Imp  LOCKRESOURCE         (KERNEL.62)
 0000:0000  Imp  __MOD_KERNEL         (KERNEL.520)
 0000:0000  Imp  __MOD_KEYBOARD       (KERNEL.526)
 0000:0000  Abs  __acrtused
 0000:0000  Imp  __MOD_SOUND          (KERNEL.527)
 0000:0000  Imp  __MOD_TOOLHELP       (KERNEL.530)
 0000:0000  Imp  IsBadHugeReadPtr     (KERNEL.346)
 0000:0000  Imp  LocalInit            (KERNEL.4)
 0000:0000  Imp  __MOD_GDI            (KERNEL.524)
 0000:0000  Imp  __MOD_WINSOCK        (KERNEL.529)
 0000:0000  Imp  GLOBALUNLOCK         (KERNEL.19)
 0000:0000  Imp  __MOD_USER           (KERNEL.522)
 0000:0000  Imp  HandleParamError     (KERNEL.327)
 0000:0000  Imp  GlobalFree           (KERNEL.17)
 0000:0000  Imp  __MOD_COMMDLG        (KERNEL.532)
 0000:0000  Imp  IsBadWritePtr        (KERNEL.335)
 0000:0000  Imp  GETMODULEFILENAME    (KERNEL.49)
 0000:0000  Imp  GlobalLock           (KERNEL.18)
 0000:0000  Imp  GlobalReAlloc        (KERNEL.16)
 0000:0000  Imp  __MOD_MMEDIA         (KERNEL.531)
 0000:0000  Imp  __MOD_DKERNEL        (KERNEL.521)
 0000:0000  Imp  __MOD_DGDI           (KERNEL.525)
 0000:0000  Imp  __MOD_SHELL          (KERNEL.528)
 0000:0000  Imp  WOW16Call            (KERNEL.500)
 0000:0000  Imp  IsBadReadPtr         (KERNEL.334)
 0000:0000  Imp  GlobalHandle         (KERNEL.21)
 0000:0000  Imp  __MOD_DUSER          (KERNEL.523)
 0000:0000  Imp  GlobalAlloc          (KERNEL.15)
 0000:0000  Imp  GETMODULEHANDLE      (KERNEL.47)
 0000:0000  Imp  IsBadHugeWritePtr    (KERNEL.347)
 0001:0000       GDI16
 0001:002F       WEP
 0001:003B       CheckStockObject
 0001:0062       IGetMetafileBits
 0001:0085       ISetMetafileBits
 0001:009B       ISetMetafileBitsBetter
 0001:00BD       ICLOSEMETAFILE
 0001:00CA       ICOPYMETAFILE
 0001:00D7       ICREATEMETAFILE
 0001:00E4       IDELETEMETAFILE
 0001:00F1       IGETMETAFILE
 0001:00FE       IENUMMETAFILE
 0001:010B       ISVALIDMETAFILE
 0001:0118       IPLAYMETAFILE
 0001:0125       IPLAYMETAFILERECORD
 0001:0132       WOWADDFONTRESOURCE
 0001:013F       IANIMATEPALETTE
 0001:014C       IARC
 0001:0159       IBITBLT
 0001:0166       BRUTE
 0001:0173       ICHORD
 0001:0180       CLOSEJOB
 0001:018D       ICOMBINERGN
 0001:019A       ICOMPATIBLEBITMAP
 0001:01A7       COPY
 0001:01B4       ICREATEBITMAP
 0001:01C1       ICREATEBITMAPINDIRECT
 0001:01CE       ICREATEBRUSHINDIRECT
 0001:01DB       ICREATECOMPATIBLEBITMAP
 0001:01E8       ICREATECOMPATIBLEDC
 0001:01F5       ICREATEDC
 0001:0202       ICREATEDIBITMAP
 0001:020F       WOWCREATEDIBPATTERNBRUSH
 0001:021C       ICREATEDISCARDABLEBITMAP
 0001:0229       CREATEELLIPTICRGN
 0001:0236       ICREATEELLIPTICRGNINDIRECT
 0001:0243       ICREATEFONT
 0001:0250       ICREATEFONTINDIRECT
 0001:025D       ICREATEHATCHBRUSH
 0001:026A       ICREATEIC
 0001:0277       ICREATEPALETTE
 0001:0284       ICREATEPATTERNBRUSH
 0001:0291       ICREATEPEN
 0001:029E       ICREATEPENINDIRECT
 0001:02AB       ICREATEPOLYGONRGN
 0001:02B8       ICREATEPOLYPOLYGONRGN
 0001:02C5       ICREATEREALBITMAP
 0001:02D2       ICREATEREALBITMAPINDIRECT
 0001:02DF       CREATERECTRGN
 0001:02EC       ICREATERECTRGNINDIRECT
 0001:02F9       CREATEROUNDRECTRGN
 0001:0306       CREATESOLIDBRUSH
 0001:0313       CREATEUSERBITMAP
 0001:0320       CREATEUSERDISCARDABLEBITMAP
 0001:032D       DEATH
 0001:033A       IDELETEABOVELINEFONTS
 0001:0347       IDELETEDC
 0001:0354       DELETEJOB
 0001:0361       IDELETEOBJECT
 0001:036E       DEVICECOLORMATCH
 0001:037B       IDEVICEMODE
 0001:0388       DMBITBLT
 0001:0395       DMCOLORINFO
 0001:03A2       DMENUMDFONTS
 0001:03AF       DMENUMOBJ
 0001:03BC       DMOUTPUT
 0001:03C9       DMPIXEL
 0001:03D6       DMREALIZEOBJECT
 0001:03E3       DMSCANLR
 0001:03F0       DMSTRBLT
 0001:03FD       DMTRANSPOSE
 0001:040A       IDPTOLP
 0001:0417       IDPXLATE
 0001:0424       IELLIPSE
 0001:0431       ENDSPOOLPAGE
 0001:043E       IENUMCALLBACK
 0001:044B       IENUMFONTS
 0001:0458       IENUMOBJECTS
 0001:0465       IEQUALRGN
 0001:0472       IESCAPE
 0001:047F       IEXCLUDECLIPRECT
 0001:048C       EXCLUDEVISRECT
 0001:0499       IEXTDEVICEMODE
 0001:04A6       IEXTFLOODFILL
 0001:04B3       IEXTTEXTOUT
 0001:04C0       FASTWINDOWFRAME
 0001:04CD       IFILLRGN
 0001:04DA       FINALGDIINIT
 0001:04E7       IFLOODFILL
 0001:04F4       IFRAMERGN
 0001:0501       GDIINIT2
 0001:050E       GDIMOVEBITMAP
 0001:051B       GDIREALIZEPALETTE
 0001:0528       GDISELECTPALETTE
 0001:0535       IGETASPECTRATIOFILTER
 0001:0542       IGETBITMAPBITS
 0001:054F       IGETBITMAPDIMENSION
 0001:055C       GETBKCOLOR
 0001:0569       GETBKMODE
 0001:0576       GETBRUSHORG
 0001:0583       IGETCHARWIDTH
 0001:0590       IGETCLIPBOX
 0001:059D       GETCLIPRGN
 0001:05AA       GETCURLOGFONT
 0001:05B7       IGETCURRENTOBJECT
 0001:05C4       GETCURRENTPOSITION
 0001:05D1       GETDCORG
 0001:05DE       GETDCSTATE
 0001:05EB       IGETDEVICECAPS
 0001:05F8       IGETDIBITS
 0001:0605       IGETENVIRONMENT
 0001:0612       GETMAPMODE
 0001:061F       IGETNEARESTCOLOR
 0001:062C       IGETNEARESTPALETTEINDEX
 0001:0639       IGETOBJECT
 0001:0646       IGETPALETTEENTRIES
 0001:0653       GETPHYSICALFONTHANDLE
 0001:0660       IGETPIXEL
 0001:066D       GETPOLYFILLMODE
 0001:067A       GETRELABS
 0001:0687       IGETREGIONDATA
 0001:0694       IGETRGNBOX
 0001:06A1       GETROP2
 0001:06AE       GETSPOOLJOB
 0001:06BB       IGETSTOCKOBJECT
 0001:06CB       GETSTRETCHBLTMODE
 0001:06D8       IGETSYSTEMPALETTEENTRIES
 0001:06E5       IGETSYSTEMPALETTEUSE
 0001:06F2       GETTEXTALIGN
 0001:06FF       IGETTEXTCHARACTEREXTRA
 0001:070C       GETTEXTCOLOR
 0001:0719       IGETTEXTEXTENT
 0001:0726       IGETTEXTFACE
 0001:0733       IGETTEXTMETRICS
 0001:0740       GETVIEWPORTEXT
 0001:074D       GETVIEWPORTORG
 0001:075A       GETWINDOWEXT
 0001:0767       GETWINDOWORG
 0001:0774       IGSV
 0001:0781       INQUIREVISRGN
 0001:078E       IINTERNALCREATEDC
 0001:079B       IINTERSECTCLIPRECT
 0001:07A8       INTERSECTVISRECT
 0001:07B5       IINVERTRGN
 0001:07C2       ISDCCURRENTPALETTE
 0001:07CF       ISDCDIRTY
 0001:07DC       ILINEDDA
 0001:07E9       ILINETO
 0001:07F6       ILPTODP
 0001:0803       ILVBUNION
 0001:0810       IMFDRAWTEXT
 0001:081D       IMOVETO
 0001:082A       IOFFSETCLIPRGN
 0001:0837       IOFFSETORG
 0001:0844       IOFFSETRGN
 0001:0851       IOFFSETVIEWPORTORG
 0001:085E       OFFSETVISRGN
 0001:086B       IOFFSETWINDOWORG
 0001:0878       OPENJOB
 0001:0885       IPAINTRGN
 0001:0892       IPATBLT
 0001:089F       IPIE
 0001:08AC       IPIXTOLINE
 0001:08B9       IPOLYGON
 0001:08C6       IPOLYLINE
 0001:08D3       IPOLYPOLYGON
 0001:08E0       IPOLYPOLYLINEWOW
 0001:08ED       IPTINREGION
 0001:08FA       IPTVISIBLE
 0001:0907       QUERYJOB
 0001:0914       IRCOS
 0001:0921       REALIZEDEFAULTPALETTE
 0001:092E       IRECTANGLE
 0001:093B       IRECTINREGION
 0001:0948       IRECTSTUFF
 0001:0955       IRECTVISIBLE
 0001:0962       WOWREMOVEFONTRESOURCE
 0001:096F       IRESIZEPALETTE
 0001:097C       IRESTOREDC
 0001:0989       RESTOREVISRGN
 0001:0996       RESURRECTION
 0001:09A3       IROUNDRECT
 0001:09B0       IRSIN
 0001:09BD       ISAVEDC
 0001:09CA       SAVEVISRGN
 0001:09D7       ISCALEEXT
 0001:09E4       ISCALEVIEWPORTEXT
 0001:09F1       ISCALEWINDOWEXT
 0001:09FE       SCANLR
 0001:0A0B       ISELECTCLIPRGN
 0001:0A18       ISELECTOBJECT
 0001:0A25       SELECTVISRGN
 0001:0A32       ISETBITMAPBITS
 0001:0A3F       ISETBITMAPDIMENSION
 0001:0A4C       ISETBKCOLOR
 0001:0A59       ISETBKMODE
 0001:0A66       ISETBRUSHORG
 0001:0A73       SETDCORG
 0001:0A80       SETDCSTATE
 0001:0A8D       SETDCSTATUS
 0001:0A9A       ISETDIBITS
 0001:0AA7       ISETDIBITSTODEVICE
 0001:0AB4       ISETENVIRONMENT
 0001:0AC1       ISETMAPMODE
 0001:0ACE       ISETMAPPERFLAGS
 0001:0ADB       ISETPALETTEENTRIES
 0001:0AE8       ISETPIXEL
 0001:0AF5       ISETPOLYFILLMODE
 0001:0B02       ISETRECTRGN
 0001:0B0F       SETRELABS
 0001:0B1C       ISETROP2
 0001:0B29       ISETSTRETCHBLTMODE
 0001:0B36       ISETSYSTEMPALETTEUSE
 0001:0B43       ISETTEXTALIGN
 0001:0B50       ISETTEXTCHARACTEREXTRA
 0001:0B5D       ISETTEXTCOLOR
 0001:0B6A       ISETTEXTJUSTIFICATION
 0001:0B77       ISETVIEWPORTEXT
 0001:0B84       ISETVIEWPORTORG
 0001:0B91       ISETWINDOWEXT
 0001:0B9E       ISETWINDOWORG
 0001:0BAB       ISETWINVIEWEXT
 0001:0BB8       SHRINKGDIHEAP
 0001:0BC5       STARTSPOOLPAGE
 0001:0BD2       ISTRETCHBLT
 0001:0BDF       ISTRETCHDIBITS
 0001:0BEC       ISTUFFINREGION
 0001:0BF9       ISTUFFVISIBLE
 0001:0C06       ITEXTOUT
 0001:0C13       IUNREALIZEOBJECT
 0001:0C20       IUPDATECOLORS
 0001:0C2D       IWORDSET
 0001:0C3A       WRITEDIALOG
 0001:0C47       WRITESPOOL
 0001:0C54       BITMAPBITS
 0001:0C61       SETDCHOOK
 0001:0C6E       GETDCHOOK
 0001:0C7B       SETHOOKFLAGS
 0001:0C88       SETBOUNDSRECT
 0001:0C95       GETBOUNDSRECT
 0001:0CA2       SELECTBITMAP
 0001:0CAF       DMEXTTEXTOUT
 0001:0CBC       DMGETCHARWIDTH
 0001:0CC9       DMSTRETCHBLT
 0001:0CD6       DMDIBBITS
 0001:0CE3       DMSTRETCHDIBITS
 0001:0CF0       DMSETDIBTODEV
 0001:0CFD       DELETESPOOLPAGE
 0001:0D0A       SPOOLFILE
 0001:0D17       ENGINEENUMERATEFONT
 0001:0D24       ENGINEDELETEFONT
 0001:0D31       ENGINEREALIZEFONT
 0001:0D3E       ENGINEGETCHARWIDTH
 0001:0D4B       ENGINESETFONTCONTEXT
 0001:0D58       ENGINEGETGLYPHBMP
 0001:0D65       ENGINEMAKEFONTDIR
 0001:0D72       IGETCHARABCWIDTHS
 0001:0D7F       IGETOUTLINETEXTMETRICS
 0001:0D8C       IGETGLYPHOUTLINE
 0001:0D99       ICREATESCALABLEFONTRESOURCE
 0001:0DA6       IGETFONTDATA
 0001:0DB3       CONVERTOUTLINEFONTFILE
 0001:0DC0       GETRASTERIZERCAPS
 0001:0DCD       ENGINEEXTTEXTOUT
 0001:0DDA       IENUMFONTFAMILIES
 0001:0DE7       IGETKERNINGPAIRS
 0001:0DF4       IRESETDC
 0001:0E01       ISTARTDOC
 0001:0E0E       IENDDOC
 0001:0E1B       ISTARTPAGE
 0001:0E28       IENDPAGE
 0001:0E35       ISETABORTPROC
 0001:0E42       IABORTDOC
 0001:0E4F       GDISEEGDIDO
 0001:0E5C       GDITASKTERMINATION
 0001:0E69       SETOBJECTOWNER
 0001:0E76       ISGDIOBJECT
 0001:0E83       MAKEOBJECTPRIVATE
 0001:0E90       FIXUPBOGUSPUBLISHERMETAFILE
 0001:0E9D       RECTVISIBLE_EHH
 0001:0EAA       RECTINREGION_EHH
 0001:0EB7       UNICODETOANSI
 0001:0EC4       IGETBITMAPDIMENSIONEX
 0001:0ED1       GETBRUSHORGEX
 0001:0EDE       GETCURRENTPOSITIONEX
 0001:0EEB       IGETTEXTEXTENTPOINT
 0001:0EF8       GETVIEWPORTEXTEX
 0001:0F05       GETVIEWPORTORGEX
 0001:0F12       GETWINDOWEXTEX
 0001:0F1F       GETWINDOWORGEX
 0001:0F2C       IOFFSETVIEWPORTORGEX
 0001:0F39       IOFFSETWINDOWORGEX
 0001:0F46       ISETBITMAPDIMENSIONEX
 0001:0F53       ISETVIEWPORTEXTEX
 0001:0F60       ISETVIEWPORTORGEX
 0001:0F6D       ISETWINDOWEXTEX
 0001:0F7A       ISETWINDOWORGEX
 0001:0F87       IMOVETOEX
 0001:0F94       ISCALEVIEWPORTEXTEX
 0001:0FA1       ISCALEWINDOWEXTEX
 0001:0FAE       IGETASPECTRATIOFILTEREX
 0001:0FBB       CREATEDIBSECTION
 0001:0FC8       GETDIBCOLORTABLE
 0001:0FD5       SETDIBCOLORTABLE
 0001:0FE2       QUERYABORT
 0001:0FF4       ValidateDIBHeader
 0001:1098       ValidateDIBSize
 0001:111A       DIB_Validate_Pointer
 0001:1140       DIB_Validate_Huge_Pointer
 0001:1167       ANIMATEPALETTE
 0001:1184       CREATEPALETTE
 0001:11B1       GETPALETTEENTRIES
 0001:11CE       GETNEARESTPALETTEINDEX
 0001:11DC       GETSYSTEMPALETTEENTRIES
 0001:11F9       GETSYSTEMPALETTEUSE
 0001:1207       RESIZEPALETTE
 0001:1215       SETPALETTEENTRIES
 0001:1232       SETSYSTEMPALETTEUSE
 0001:1240       UPDATECOLORS
 0001:124E       ABORTDOC
 0001:125F       ENDPAGE
 0001:1270       ENDDOC
 0001:1281       STARTDOC
 0001:129E       STARTPAGE
 0001:12AC       SETABORTPROC
 0001:12C6       CREATECOMPATIBLEDC
 0001:12D4       CREATEIC
 0001:1306       CREATEDC
 0001:1376       DELETEDC
 0001:1384       RESTOREDC
 0001:1392       SAVEDC
 0001:13A0       RESETDC
 0001:13EA       DELETEOBJECT
 0001:13F8       CREATEPEN
 0001:1414       CREATEPENINDIRECT
 0001:142E       CREATEHATCHBRUSH
 0001:144A       CREATEPATTERNBRUSH
 0001:1458       CREATEBRUSHINDIRECT
 0001:1472       CREATEBITMAP
 0001:148C       CREATEBITMAPINDIRECT
 0001:14CD       CREATECOMPATIBLEBITMAP
 0001:14DB       CREATEDISCARDABLEBITMAP
 0001:14E9       CREATEFONT
 0001:1511       CREATEFONTINDIRECT
 0001:152B       CREATEDIBPATTERNBRUSH
 0001:1580       SETBITMAPDIMENSION
 0001:158E       SETBITMAPDIMENSIONEX
 0001:15A8       GETBITMAPDIMENSION
 0001:15B6       GETBITMAPDIMENSIONEX
 0001:15D0       SETTEXTJUSTIFICATION
 0001:15DE       SETTEXTCHARACTEREXTRA
 0001:15EC       COPYMETAFILE
 0001:160C       CREATEMETAFILE
 0001:1626       CLOSEMETAFILE
 0001:1634       DELETEMETAFILE
 0001:1642       PLAYMETAFILE
 0001:1650       GETMETAFILE
 0001:166A       PLAYMETAFILERECORD
 0001:1690       ENUMMETAFILE
 0001:16A7       GETMETAFILEBITS
 0001:16B5       SETMETAFILEBITS
 0001:16C3       SETMETAFILEBITSBETTER
 0001:16D1       DPTOLP
 0001:16EE       LPTODP
 0001:170B       CREATEELLIPTICRGNINDIRECT
 0001:1725       CREATEPOLYGONRGN
 0001:1755       CREATEPOLYPOLYGONRGN
 0001:178E       ELLIPSE
 0001:179C       ARC
 0001:17AA       PIE
 0001:17B8       CHORD
 0001:17C6       ROUNDRECT
 0001:17D4       RECTANGLE
 0001:17E2       FLOODFILL
 0001:17F0       EXTFLOODFILL
 0001:180C       ESCAPE
 0001:1835       ENUMOBJECTS
 0001:185F       ENUMFONTS
 0001:1882       ENUMFONTFAMILIES
 0001:18A5       GETCHARWIDTH
 0001:18D8       GETPIXEL
 0001:18E6       SETPIXEL
 0001:18F8       GETSTOCKOBJECT
 0001:1914       GETBITMAPBITS
 0001:192E       GETDEVICECAPS
 0001:193C       SETBITMAPBITS
 0001:1956       GETOBJECT
 0001:1970       GETASPECTRATIOFILTER
 0001:197E       GETASPECTRATIOFILTEREX
 0001:1998       SETMAPPERFLAGS
 0001:19BD       GETNEARESTCOLOR
 0001:19CB       OFFSETVIEWPORTORG
 0001:19D9       OFFSETVIEWPORTORGEX
 0001:19F3       OFFSETWINDOWORG
 0001:1A01       OFFSETWINDOWORGEX
 0001:1A1B       SETMAPMODE
 0001:1A3C       SETWINDOWEXT
 0001:1A4A       SETWINDOWEXTEX
 0001:1A64       SETVIEWPORTEXT
 0001:1A72       SETVIEWPORTEXTEX
 0001:1A8C       SCALEVIEWPORTEXT
 0001:1A9A       SCALEVIEWPORTEXTEX
 0001:1AB4       SCALEWINDOWEXT
 0001:1AC2       SCALEWINDOWEXTEX
 0001:1ADC       GETRGNBOX
 0001:1AF6       GETTEXTEXTENT
 0001:1B10       GETTEXTEXTENTPOINT
 0001:1B36       GETTEXTCHARACTEREXTRA
 0001:1B44       GETTEXTFACE
 0001:1B6E       GETTEXTMETRICS
 0001:1B88       GETENVIRONMENT
 0001:1BBE       SETENVIRONMENT
 0001:1BE4       ADDFONTRESOURCE
 0001:1BFB       REMOVEFONTRESOURCE
 0001:1C12       CREATESCALABLEFONTRESOURCE
 0001:1C44       GETGLYPHOUTLINE
 0001:1CA5       GETFONTDATA
 0001:1CE0       GETCHARABCWIDTHS
 0001:1D13       GETOUTLINETEXTMETRICS
 0001:1D2D       GETKERNINGPAIRS
 0001:1D4B       LINETO
 0001:1D59       MOVETO
 0001:1D67       MOVETOEX
 0001:1D81       POLYLINE
 0001:1D9E       LINEDDA
 0001:1DB5       POLYGON
 0001:1DD2       POLYPOLYGON
 0001:1DF8       POLYPOLYLINEWOW
 0001:1E1E       STRETCHBLT
 0001:1E2C       BITBLT
 0001:1E3A       PATBLT
 0001:1E48       SETBRUSHORG
 0001:1E56       UNREALIZEOBJECT
 0001:1E64       EXCLUDECLIPRECT
 0001:1E72       GETCLIPBOX
 0001:1E8C       INTERSECTCLIPRECT
 0001:1E9A       SELECTCLIPRGN
 0001:1EA8       CREATERECTRGNINDIRECT
 0001:1EC2       EQUALRGN
 0001:1ED0       RECTINREGION
 0001:1EEA       RECTVISIBLE
 0001:1F04       OFFSETRGN
 0001:1F12       OFFSETCLIPRGN
 0001:1F20       COMBINERGN
 0001:1F41       SETRECTRGN
 0001:1F4F       FILLRGN
 0001:1F5D       PTINREGION
 0001:1F6B       PAINTRGN
 0001:1F79       PTVISIBLE
 0001:1F87       FRAMERGN
 0001:1F95       INVERTRGN
 0001:1FA3       SELECTOBJECT
 0001:1FB1       SETTEXTCOLOR
 0001:1FBF       SETBKCOLOR
 0001:1FCF       SETBKMODE
 0001:1FF0       SETTEXTALIGN
 0001:200C       SETROP2
 0001:202D       SETSTRETCHBLTMODE
 0001:204E       SETPOLYFILLMODE
 0001:206F       SETWINDOWORG
 0001:207D       SETWINDOWORGEX
 0001:2097       SETVIEWPORTORG
 0001:20A5       SETVIEWPORTORGEX
 0001:20BF       SETDIBITS
 0001:211F       CREATEDIBITMAP
 0001:21B7       SETDIBITSTODEVICE
 0001:223D       GETDIBITS
 0001:229D       STRETCHDIBITS
 0001:22FA       EXTTEXTOUT
 0001:233A       TEXTOUT
 0001:2354       VStartTEXT
 0001:2354       GHANDLE0TEXT
 0001:2358       GHANDLETEXT
 0001:236C       LPFN0TEXT
 0001:2372       LPFNTEXT
 0001:238C       Inval_Param_TEXT
 0001:2394       LP0TEXT
 0001:239A       LPTEXT
 0001:23AA       CLP0TEXT
 0001:23B0       CLPTEXT
 0001:23BE       CLPexitTEXT
 0001:23C7       LPBUF0TEXT
 0001:23CD       LPBUFTEXT
 0001:23F6       LPBUFexitTEXT
 0001:2420       CLPSTRATOM0TEXT
 0001:2422       CLPSTRATOMTEXT
 0001:242E       CLPSZ0TEXT
 0001:2434       CLPSZTEXT
 0001:2455       ErrorStrPtrTEXT
 0001:245B       SETEMPTYTEXT
 0001:246C       MULDIV
 0001:246C       VEndTEXT
 0001:24D4       IAddFontResource
 0001:2594       IRemoveFontResource
 0001:2614       ICreateDIBPatternBrush
 0001:265E       __GP
 0001:269E       farGDIGlobalAlloc
 0001:26BF       CREATEPQ
 0001:2709       INSERTPQ
 0001:27A2       TestShuffle
 0001:27C4       MINPQ
 0001:27C7       EXTRACTPQ
 0001:27C9       GetMinPQ
 0001:2885       GetLesserChild
 0001:2899       DELETEPQ
 0001:28AF       SIZEPQ
 0002:0044       FTRAPPING0

Program entry point at 0001:0000
